:020000020000FC
:100000000C94AD1F18951895189518951895189576
:100010001895189518951895189518951895189578
:100020001895189518951895189518951895189568
:100030001895189518951895189518951895189558
:100040001895189518951895189518951895189548
:100050000C94860518951895189518951895189567
:10006000189518950C945309189518951895189586
:100070001895189518951895189518951895189518
:100080001895189518951895189518951895189508
:1000900018951895189518951895189518951895F8
:1000A00018951895189518951895189518951895E8
:1000B00018951895189518951895189518951895D8
:1000C00018951895189518951895189518951895C8
:1000D00018951895189518951895189518951895B8
:1000E00018951895189518951895189518951895A8
:1000F0001895189518951895189518951895189598
:100100001895189518951895189518951895189587
:100110001895189518951895189518950C947505B7
:100120001895189518951895189518951895189567
:10013000189518950C94F704189518951895189516
:100140001895189518951895189518951895189547
:100150001895189518951895189518951895189537
:100160001895189518951895189518951895189527
:100170001895189518951895189518951895189517
:100180001895189518951895189518951895189507
:1001900018951895189518951895189518951895F7
:1001A00018951895189518951895189518951895E7
:1001B00018951895189518951895189518951895D7
:1001C00018951895189518951895189518951895C7
:1001D00018951895189518951895189518951895B7
:1001E00018951895189518951895189518951895A7
:1001F000189518951895189518951895AA594EBEE2
:1002000034D514BEAE16863CF81D473E59298B3EA8
:10021000F81D473EAE16863C34D514BEAA594EBED4
:10022000D4D26FBCBB3CF2BC872453BD1A6DA4BDB5
:10023000AE76E6BD17740FBEB5875B3F17740FBE71
:10024000AE76E6BD1A6DA4BD872453BDBB3CF2BC9F
:10025000D4D26FBC14BEA1BD6FEDFCBDDC252FBE9A
:10026000E9383F3FDC252FBE6FEDFCBD14BEA1BDBC
:10027000010102040804040201012A2A2A2A2A2A66
:030280002A2A2AFD
:1002840000017126702645452602382611B1250B3A
:10029400762501CA2501452601432601382602CACE
:1002A4002505632501A42501B125037F2502B12578
:1002B40003AD25FB0BEC0093520008E000935000C3
:1002C400E1E5F0E0008103FFFBCF03EC0093550070
:1002D400E0E5F0E0008100610083E1E5F0E0008109
:1002E40004FFFBCF08ED04BF04E000934000E0E509
:1002F400F0E000810E7F0083089501E0009328025E
:1003040000E300932902089501E00093300208E31A
:100314000093310208950DE00093200300E400935C
:10032400210300E00093220300E40093240300EE81
:100334000093280300EE00932A0300EE00932A039F
:1003440008950150104098018901232BD1F7089595
:100354008A93802F03C008EE1DEFF3DF8A95082FE0
:10036400802F0023C1F7899108950E942B2380E0F8
:1003740090E0A0E0B0E048E0442E1BC0442D50E0E3
:10038400440F551F440F551FFA01E658FE4D0080D7
:10039400118022803380442D50E0440F551F440FB8
:1003A400551FFA01E258FE4D0082118222823382E7
:1003B4004A9441E0441610F7EEE7F1E2008311831A
:1003C40022833383442423C0042D10E0000F111F23
:1003D400000F111FF801E450FE4F459155916591AE
:1003E4007491042D10E0000F111F000F111FF8016C
:1003F400E258FE4D00811181228133810E94B02197
:10040400AC01BD010E944F21C801D901439409E008
:100414004016D0F28C019D01E5E00C943C230E942F
:100424002B2380E090E0A0E0B0E048E0442E1BC025
:10043400442D50E0440F551F440F551FFA01E25656
:10044400FE4D0080118022803380442D50E0440F03
:10045400551F440F551FFA01EE55FE4D00821182BF
:10046400228233824A9441E0441610F7E2EAF1E230
:100474000083118322833383442423C0042D10E09A
:10048400000F111F000F111FF801E450FE4F45919A
:10049400559165917491042D10E0000F111F000F08
:1004A400111FF801EE55FE4D008111812281338127
:1004B4000E94B021AC01BD010E944F21C801D901A5
:1004C400439409E04016D0F28C019D01E5E00C94C0
:1004D4003C230E942B2380E090E0A0E0B0E04CE0BD
:1004E400442E1BC0442D50E0440F551F440F551F8C
:1004F400FA01EE53FE4D0080118022803380442D9A
:1005040050E0440F551F440F551FFA01EA53FE4DA6
:1005140000821182228233824A9441E0441610F709
:10052400E6ECF1E20083118322833383442423C065
:10053400042D10E0000F111F000F111FF801E05EE1
:10054400FD4F4591559165917491042D10E0000F74
:10055400111F000F111FF801EA53FE4D0081118194
:10056400228133810E94B021AC01BD010E944F2140
:10057400C801D90143940DE04016D0F28C019D01CD
:10058400E5E00C943C230E942B2380E090E0A0E063
:10059400B0E04CE0442E1BC0442D50E0440F551FE6
:1005A400440F551FFA01EA50FE4D0080118022804D
:1005B4003380442D50E0440F551F440F551FFA015A
:1005C400E650FE4D00821182228233824A9441E039
:1005D400441610F7EAEFF1E2008311832283338398
:1005E400442423C0042D10E0000F111F000F111F1D
:1005F400F801E05EFD4F4591559165917491042D8C
:1006040010E0000F111F000F111FF801E650FE4DFE
:1006140000811181228133810E94B021AC01BD018E
:100624000E944F21C801D90143940DE04016D0F235
:100634008C019D01E5E00C943C230E942B2380E077
:1006440090E0A0E0B0E046E0442E1BC0442D50E012
:10065400440F551F440F551FFA01E65DFD4D008000
:10066400118022803380442D50E0440F551F440FE5
:10067400551FFA01E25DFD4D008211822282338210
:100684004A9441E0441610F7EEE2F2E2008311834B
:1006940022833383442423C0042D10E0000F111F50
:1006A400000F111FF801EC5AFD4F459155916591CA
:1006B4007491042D10E0000F111F000F111FF80199
:1006C400E25DFD4D00811181228133810E94B021C0
:1006D400AC01BD010E944F21C801D901439407E038
:1006E4004016D0F28C019D01E5E00C943C230E945D
:1006F4002B2380E090E0A0E0B0E046E0442E1BC055
:10070400442D50E0440F551F440F551FFA01EA5B76
:10071400FD4D0080118022803380442D50E0440F31
:10072400551F440F551FFA01E65BFD4D00821182EF
:10073400228233824A9441E0441610F7EAE4F2E25A
:100744000083118322833383442423C0042D10E0C7
:10075400000F111F000F111FF801EC5AFD4F4591B6
:10076400559165917491042D10E0000F111F000F35
:10077400111FF801E65BFD4D008111812281338157
:100784000E94B021AC01BD010E944F21C801D901D2
:10079400439407E04016D0F28C019D01E5E00C94EF
:1007A4003C239A938A93842F682F70E0660F771FF7
:1007B400660F771FFB01EA59FD4D008011802280EE
:1007C40033800019110922093309052E1124A001CF
:1007D40060E070E00E948E20482F50E0440F551FC7
:1007E400440F551FFA01EA59FD4D40815181628140
:1007F4007381040F151F261F371F90E0880F991F60
:10080400880F991FFC01EA59FD4D0083118322834F
:1008140033838991999108951091480001E00093E0
:1008240048002091A0003091A2000091A2000C7F0A
:1008340004600093A2004FB77894E8E4F0E00081EC
:10084400016000835091CD01EF93FF930F932F9399
:10085400EBECF1E008ED21E004BF20832F910F9130
:10086400FF91EF9103E00093CD0188951093480028
:100874002093A0003093A2005093CD014FBF089560
:10088400EFECF1E0008107FDFBCF0895F9DFEFEC19
:10089400F1E0008101FF11C006E30093CA01EF9368
:1008A400FF930F932F93EBECF1E008ED21E004BFED
:1008B40020832F910F91FF91EF9108959A938A933A
:1008C400C801DEDFFC01E05CF140B89750F44091D0
:1008D400232450E009E010E00E94FB1F800F911FC9
:1008E40017C0803901E0900798F44091222450E029
:1008F40000E210E00E94FB1F98014091232450E085
:1009040000E610E00E94FB1F200F311F820F931F8F
:10091400082F0093C001892F8F718093C10100E0DB
:100924000093C20106E00093CA01EF93FF930F9373
:100934002F93EBECF1E008ED21E004BF20832F912D
:100944000F91FF91EF910091C401899199910895BC
:100954000E942D23C801A22F00E00093060900E0A5
:1009640000934608FC01E05CF140B89750F44091D4
:10097400232450E009E010E00E94FB1F800F911F28
:1009840017C0803901E0900798F44091222450E088
:1009940000E210E00E94FB1F98014091232450E0E4
:1009A40000E610E00E94FB1F200F311F820F931FEF
:1009B4006DDF03E30093CA01082F0093C001892F60
:1009C4008F718093C10100E00093C201A093C40120
:1009D40005E30093CA0120DF03E00093060901E068
:1009E40000934608E3E00C943E239A938A93FA9387
:1009F400EA930A927A936A935A934A933A932A937C
:100A04001A930A930FB60091EA2303950770009393
:100A1400EA230091EA2310E0000F111FF801E353C9
:100A2400FD4D0081118100933A0310933B03009123
:100A3400EA2310E0000F111FF801E354FD4D00817B
:100A440011810093380310933903E0E0F2E0008150
:100A5400046000830091EC230023B1F100915D2335
:100A640010915E23212F220F220B322F4091EA2373
:100A740050E0440F551F440F551FFA01E35EFC4D2F
:100A84004081518162817381400F511F621F731F26
:100A9400408351836283738380916E2390916F238B
:100AA400019680936E2390936F230091702310918D
:100AB40071238017910741F400E00093EC2310E0C8
:100AC40000936E2310936F230FBE099119912991FE
:100AD400399149915991699179910990E991F991E3
:100AE4008991999118952A931A930A932FB7009193
:100AF40010021091110200935D2310935E232FBF07
:100B040009911991299118955A924A92BA93AA93E4
:100B14009A938A93FA93EA933A922A921A920A92AD
:100B24007A936A935A934A933A932A931A930A9319
:100B34005FB60091EC23002309F09DC38091E62366
:100B44009091E72301968093E6239093E7238E31D7
:100B540000E0900719F400E0009325248091E42339
:100B64009091E52301968093E4239093E5238037C5
:100B740007E1900749F400E010E00093E4231093A8
:100B8400E52301E0009306240091E4230F7701306C
:100B940019F401E000930D2480E036C05091F22353
:100BA400482F642F082F10E0000F111F000F111F92
:100BB400F801E35EFC4D0081118122813381409173
:100BC400F3230E946320462FECDD482F50E0440FAE
:100BD400551F440F551FFA01E35CFC4D008311833C
:100BE4002283338300E010E020E030E0482F50E01F
:100BF400440F551F440F551FFA01E35EFC4D00835B
:100C04001183228333838395883040F20FEF00935E
:100C1400EC2300E010E020E030E0EEE7F3E20083B4
:100C2400118322833383EAE7F3E20083118322836F
:100C3400338300E010E020E030E0EEE1F4E20083F2
:100C4400118322833383442495C0042D10E0000FC4
:100C5400111F000F111FF801E35CFC4D408151810D
:100C640062817381042D10E0000F111F000F111F0A
:100C7400F801E35CFC4D00811181228133810E94E3
:100C84003B200E94F020EEE1F4E240815181628138
:100C940073810E944F21EEE1F4E2008311832283E9
:100CA4003383EAE7F3E200811181228133810E94D8
:100CB400F020C801D901042D10E0000F111F000F0E
:100CC400111FF801E35CFC4D008111812281338105
:100CD4000E94F020442D50E0440F551F440F551F2F
:100CE400FA01E352FD4D40815181628173810E947A
:100CF400B021AC01BD010E944F210E94FD20EAE712
:100D0400F3E20083118322833383EEE7F3E200816D
:100D14001181228133810E94F020C801D901042D60
:100D240010E0000F111F000F111FF801E35CFC4DD0
:100D340000811181228133810E94F020442D50E0F2
:100D4400440F551F440F551FFA01E350FD4D4081D8
:100D54005181628173810E94B021AC01BD010E9466
:100D64004F210E94FD20EEE7F3E2008311832283EA
:100D74003383439408E0401608F467CF40E050E022
:100D840060E071E4EEE1F4E20081118122813381BB
:100D94000E9429220E944929EEE1F4E20083118392
:100DA40022833383009174231091752320E030E073
:100DB4000E94FB20A801B901EEE1F4E20081118157
:100DC400228133810E9429220E94FD2000936C23FA
:100DD40010936D230091F32310E0F801EA58FD4FBE
:100DE400449150E000916C2310916D230E940F20D8
:100DF40000936C2310936D230091E82310E0F80115
:100E0400E059FD4F449150E000916C2310916D2303
:100E14000E940F2000936C2310936D230091E8230C
:100E2400002351F400916C2310916D23000F111FC6
:100E340000936C2310936D23EAE7F3E200811181A0
:100E440022813381EAE8F3E200831183228333832E
:100E5400EEE7F3E20081118122813381EEE8F3E2CF
:100E64000083118322833383E6E9F3E20081118155
:100E740022813381EAE8F3E2408151816281738106
:100E840004171507260737077CF4E6E9F3E2008127
:100E94001181228133810F5F1F4F2F4F3F4F0083FA
:100EA4001183228333830EC0E6E9F3E200811181CA
:100EB400228133810150104020403040008311834F
:100EC40022833383E2E9F3E20081118122813381B9
:100ED400EEE8F3E2408151816281738104171507C2
:100EE400260737077CF4E2E9F3E2008111812281CD
:100EF40033810F5F1F4F2F4F3F4F00831183228396
:100F040033830EC0E2E9F3E200811181228133814F
:100F140001501040204030400083118322833383EA
:100F24000091EB230023D9F000E00093EB23EAE8DF
:100F3400F3E20081118122813381E6E9F3E2008347
:100F4400118322833383EEE8F3E20081118122814D
:100F54003381E2E9F3E20083118322833383E6E9F8
:100F6400F3E20081118122813381EAE8F3E24081D6
:100F7400518162817381401B510B620B730B40835F
:100F8400518362837383E2E9F3E200811181228158
:100F94003381EEE8F3E24081518162817381401B29
:100FA400510B620B730B4083518362837383EAE8B2
:100FB400F3E20081118122813381E2ECF3E20083C8
:100FC400118322833383EEE8F3E2008111812281CD
:100FD4003381E6ECF3E200831183228333830091AF
:100FE400EE23013009F077C00091FD23013029F58B
:100FF400EAE8F3E200811181228133810E94F0202A
:101004000E94B7010E94FD20E2EBF3E2008311830A
:1010140022833383EEE8F3E200811181228133815C
:101024000E94F0200E9411020E94FD20E6EBF3E2F0
:10103400008311832283338366C00091FD23023031
:1010440029F5EAE8F3E200811181228133810E94CB
:10105400F0200E946B020E94FD20E2EBF3E2008389
:10106400118322833383EEE8F3E20081118122812C
:1010740033810E94F0200E94C5020E94FD20E6EB0D
:10108400F3E200831183228333833DC0EAE8F3E271
:1010940000811181228133810E94F0200E941F036C
:1010A4000E94FD20E2EBF3E2008311832283338369
:1010B400EEE8F3E200811181228133810E94F02065
:1010C4000E9479030E94FD20E6EBF3E20083118382
:1010D4002283338318C0EAE8F3E20081118122817C
:1010E4003381E2EBF3E20083118322833383EEE85E
:1010F400F3E20081118122813381E6EBF3E2008384
:10110400118322833383E2EBF3E200811181228194
:101114003381EAEBF3E24081518162817381400FB4
:10112400511F621F731F4083518362837383E6EBF5
:10113400F3E20081118122813381EEEBF3E24081FD
:10114400518162817381400F511F621F731F40835D
:10115400518362837383E2ECF3E200811181228183
:101164003381EAECF3E24081518162817381400F63
:10117400511F621F731F4083518362837383E6ECA4
:10118400F3E20081118122813381EEECF3E24081AC
:10119400518162817381400F511F621F731F40830D
:1011A4005183628373830091032403950093032482
:1011B40010910024101708F05EC000E0009303248F
:1011C400EAEBF3E20081118122813381E2E8F3E268
:1011D400008311832283338300E010E020E030E0B9
:1011E400EAEBF3E20083118322833383EEEBF3E231
:1011F4000081118122813381E6E8F3E200831183C7
:101204002283338300E010E020E030E0EEEBF3E2F1
:101214000083118322833383EAECF3E2008111819A
:1012240022813381E2EDF3E200831183228333834D
:1012340000E010E020E030E0EAECF3E20083118308
:1012440022833383EEECF3E2008111812281338126
:10125400E6EDF3E2008311832283338300E010E0A0
:1012640020E030E0EEECF3E2008311832283338349
:1012740001E00093F9235FBE0991199129913991F5
:1012840049915991699179910990199029903990CE
:10129400E991F99189919991A991B99149905990BC
:1012A40018954A92BA93AA939A938A93FA93EA93D3
:1012B4003A922A921A920A927A936A935A934A9386
:1012C4003A932A931A930A934FB600E010E00093DE
:1012D4001224109313248091A008813489F4E5E248
:1012E400F4E200810160008300E010E00093E62353
:1012F4001093E723E4E6F6E0008102600083BFC5B3
:1013040000912524002309F4BAC500912524033053
:1013140031F400912524002309F018C4B0C58434A5
:10132400F9F401E2D9D500916123DED50091692356
:10133400DBD5E2E8F3E20081118145E00E94092057
:10134400D3D5E6E8F3E20081118145E00E9409204B
:10135400CBD500910B24C8D500E000932524D9CF28
:10136400833571F40091F5230A950093F523002346
:1013740019F401E00093F52300E000932524C9CF7C
:10138400843571F40091F52303950093F523053119
:1013940018F004E10093F52300E000932524B9CF6D
:1013A400863471F40091FD2303950093FD230430EA
:1013B40018F001E00093FD2300E000932524A9CF59
:1013C400873509F05FC00E94C01501E285D50E94EF
:1013D40034128AD54FE050E000916C2310916D23B4
:1013E4000E940F2081D50091FD237ED50091F52325
:1013F4007BD50091FC2378D500916A2375D50091A3
:10140400232472D5009122246FD5009107246CD532
:10141400E0915F23F09160233196AF01652F660F51
:10142400660B762F00E81DE82BE530E00E948E2045
:10143400009318241093192400911824109119244E
:101444001A930A9324E231E206EA12E20E942E2958
:10145400229606EA12E228D501EF11E02FDA44D5EC
:1014640000916B2341D500916C2310916D23083EAC
:1014740023E0120718F401E00093EB2300E000934B
:10148400252447CF853409F06DC00E94C01501E2C0
:1014940023D50091232428D50091222425D5009119
:1014A400072422D50091F2231FD5009104241CD5D2
:1014B4000091E82319D50091F32316D50091002457
:1014C40013D50091FE2310D50091ED230DD5009185
:1014D400FF230AD50091F42307D50091F62304D500
:1014E4000091092401D500910824FED4E0915F23E2
:1014F400F09160233196AF01652F660F660B762F4E
:1015040000E81DE82BE530E00E948E2000931824AB
:101514001093192400911824109119241A930A93F2
:1015240024E231E206EA12E20E942E29229606EA19
:1015340012E2BAD4EFE3F1E2008111812281338116
:101544003A932A931A930A9329E231E206EA12E2C1
:101554000E942E29249606EA12E2A6D400E0009303
:101564002524D7CE8B3299F400916623BDD4009103
:101574006723BAD44FE050E000916C2310916D239F
:101584000E940F20B1D400E000932524C2CE8F36F0
:1015940049F4E4E8F6E000810B7F008300E0009367
:1015A4002524B7CE893709F043C001E295D40091D0
:1015B40023249AD40091222497D40091072494D40C
:1015C400E0915F23F09160233196AF01652F660FA0
:1015D400660B762F00E81DE82BE530E00E948E2094
:1015E400009318241093192400911824109119249D
:1015F4001A930A9324E231E206EA12E20E942E29A7
:10160400229606EA12E250D40091DA231091DB23E9
:101614001A930A932EE231E206EA12E20E942E297C
:10162400229606EA12E240D400E00093252471CE0B
:10163400853741F5E0915F23F09160233196AF0146
:10164400652F660F660B762F00E81DE82BE530E06A
:101654000E948E20009318241093192400911824BA
:10166400109119241A930A9324E231E206EA12E251
:101674000E942E29229606EA12E216D400E0009374
:10168400252447CE893631F4ACD62ED400E000931D
:1016940025243FCE813779F40091EE23013021F4E3
:1016A40000E00093EE2303C001E00093EE2300E08A
:1016B400009325242ECE823671F4009144060F70D7
:1016C40000934406E4E6F6E000810D7F008300E029
:1016D400009325241ECE803579F408E00093A408F5
:1016E4000FE00E94AA0108E10093A4088091A008D9
:1016F40000E0009325240DCE853649F4009124069C
:1017040003600093240600E00093252402CE823770
:1017140049F4009124060C7F0093240600E0009312
:101724002524F7CD8636C1F5EFE5F3E2008111817A
:10173400015010400083118300915F2310916023B6
:101744000093260910932709E0915F23F091602309
:101754003196AF01652F660F660B762F00E81DE802
:101764002BE530E00E948E20009318241093192456
:1017740000911824109119241A930A9324E231E257
:1017840006EA12E20E942E29229606EA12E28CD37D
:1017940000E000932524BDCD8736C1F5EFE5F3E2E3
:1017A400008111810F5F1F4F0083118300915F231C
:1017B400109160230093260910932709E0915F2379
:1017C400F09160233196AF01652F660F660B762F7B
:1017D40000E81DE82BE530E00E948E2000931824D9
:1017E4001093192400911824109119241A930A9320
:1017F40024E231E206EA12E20E942E29229606EA47
:1018040012E252D300E00093252483CD883649F5B3
:10181400ECD3E0915F23F09160233196AF01652F03
:10182400660F660B762F00E81DE82BE530E00E947A
:101834008E200093182410931924009118241091D9
:1018440019241A930A9324E231E206EA12E20E946E
:101854002E29229606EA12E227D300E000932524DB
:1018640058CD8B3631F5E091DA23F091DB233197B3
:10187400E093DA23F093DB23FF2332F408E611E04C
:101884000093DA231093DB234DD60091DA231091D1
:10189400DB231A930A932EE231E206EA12E20E9453
:1018A4002E29229606EA12E2FFD200E000932524B4
:1018B40030CD8A3641F5E091DA23F091DB2331967D
:1018C400E093DA23F093DB23E83601E0F00734F009
:1018D40000E010E00093DA231093DB2323D6009179
:1018E400DA231091DB231A930A932EE231E206EAFB
:1018F40012E20E942E29229606EA12E2D5D200E0D4
:101904000093252406CD8C36A9F4A8D30091DA23BC
:101914001091DB231A930A9323E331E206EA12E2DD
:101924000E942E29229606EA12E2BED200E000931B
:101934002524EFCC873759F40E94C0150091072461
:10194400023009F4DCD200E000932524E2CC843692
:1019540041F507E00093F22301E00093042406E03C
:101964000093FF2301E00093E82301E00093F323B5
:1019740002E00093FE2301E00093002401E00093C1
:10198400ED2301E00093F4230FE00093F52308E036
:101994000093F62308E50093092400E0009325242E
:1019A400B8CC823579F42FEF0AEF11E00E94AA0433
:1019B40000E21EE40E94A30108ED04BF01E00093CD
:1019C4007900A7CC813339F401E00093FA2300E0D5
:1019D400009325249ECC823311F500E010E000939F
:1019E400E2231093E3230093E0231093E12320E008
:1019F40000E110E00E94AA0420E001E110E00E944E
:101A0400AA042091E2233091E3230091E023109172
:101A1400E1230E94011600E0009325247ACC893347
:101A240081F5009109240395009309240B3518F0DE
:101A34000AE5009309240091092410E01195019509
:101A44001040212F220F220B322F0E94F02043E35B
:101A540053E365E672E40E9429220E94BE29A8018C
:101A6400B90100E010E020E83FE30E942922EFE3FF
:101A7400F1E2008311832283338300E00093252461
:101A840048CC883381F5009109240A9500930924F0
:101A9400063418F406E4009309240091092410E0A4
:101AA400119501951040212F220F220B322F0E94F5
:101AB400F02043E353E365E672E40E9429220E9486
:101AC400BE29A801B90100E010E020E83FE30E942C
:101AD4002922EFE3F1E2008311832283338300E0C0
:101AE4000093252416CC873359F5D7D70BEE11E094
:101AF4000E946004B02FA0E00CEE11E00E9460048C
:101B040010E0A02BB12BA0937823B09379230091FC
:101B14007823109179231A930A9329E331E206EA90
:101B240012E20E942E29229606EA12E2BDD103EFA8
:101B340011E00E946004D8D100E000932524E9CB91
:101B440003E0009325248093242499C10091242444
:101B5400063349F4282F0DEE11E00E94AA0400E098
:101B6400009325248CC1009124240533B9F503EF97
:101B740011E00E94600410E00093182410931924CB
:101B8400E0911824F0911924369734F008ED04BF3D
:101B940001E00093790073C1282F0EEE11E00E943A
:101BA400AA040E94C015009107249ED120911824F4
:101BB400239503EF11E00E94AA042091E4230BEF84
:101BC40011E00E94AA040E94C827202F0AEE11E007
:101BD4000E94AA0400E00093252451C1009124240A
:101BE400063531F48093FC2300E00093252447C19B
:101BF400009124240A3579F480936A2380916A231E
:101C040090E08857904080936A0990936B0900E0B4
:101C14000093252434C100912424093481F48031B3
:101C240050F48093FF234091FF2350E008E710E035
:101C34000E94FB1FDFD200E00093252420C1009105
:101C44002424073459F4853028F48093E823009140
:101C5400E823BED600E00093252411C1009124247A
:101C6400003781F480932324209123240AEF11E088
:101C74000E94AA0400E000932524BAD600E0009351
:101C84002524FDC000912424033759F58093222490
:101C9400282F0DEF11E00E94AA04882331F400914B
:101CA400640608610093640614C0813059F4E4E6C4
:101CB400F6E000810F7E0083E4E6F6E00081086030
:101CC400008307C0823029F400916406077E0093E4
:101CD400640600E0009325248BD600E000932524BD
:101CE400CEC000912424083441F48B3010F4809346
:101CF400F22300E000932524C2C00091242403367B
:101D040041F4843010F48093042400E000932524EB
:101D1400B6C0009124240A3741F4833010F4809330
:101D2400F32300E000932524AAC0009124240D3459
:101D340041F4843010F48093002400E000932524BF
:101D44009EC000912424023441F4853010F4809321
:101D5400FE2300E00093252492C000912424013640
:101D640041F4833010F48093ED2300E000932524A4
:101D740086C000912424043761F4883010F48093E1
:101D8400F4230091F4230E943E1700E000932524DD
:101D940076C000912424083741F48A3010F48093EB
:101DA400F62300E0009325246AC0009124240D3614
:101DB40061F490E0880F991F8093DA239093DB23DA
:101DC400B1D300E0009325245AC0009124240D339C
:101DD40009F052C08093082400910824002319F5C7
:101DE4000091092410E0119501951040212F220F34
:101DF400220B322F0E94F02043E353E365E672E4A2
:101E04000E9429220E94BE29A801B90100E010E025
:101E140020E83FE30E942922EFE3F1E200831183EB
:101E2400228333831FC000916723102F110F110BDE
:101E3400212F312F0E94F02043E353E365E672E43F
:101E44000E9429220E94BE29A801B90100E010E0E5
:101E540020E83FE30E942922EFE3F1E200831183AB
:101E6400228333832091082405EF11E00E94AA0401
:101E740000E00093252403C000E0009325244FBE16
:101E840009911991299139914991599169917991BE
:101E94000990199029903990E991F9918991999132
:101EA400A991B991499018950E942C23C801A0E0EA
:101EB40007C0B0E0FC01EA0FFB1F008115D0A39519
:101EC400B0E0FC01EA0FFB1F0081002311F0AD30EC
:101ED40080F3E4E00C943D23E1EAF8E0108115FF7F
:101EE400FBCF0093A0080895013209F400E4E1EA6D
:101EF400F8E0108115FFFBCF0093A00808953091FE
:101F04006023232F01E010E00E94AA0420915F23A4
:101F140002E010E00E94AA043091DB23232F05E0A5
:101F240010E00E94AA042091DA2306E010E00E9447
:101F3400AA042091F2230DE110E00E94AA0420914A
:101F440004240BE110E00E94AA042091FF230CE07A
:101F540010E00E94AA042091E82304E110E00E940A
:101F6400AA042091F3230EE110E00E94AA04209118
:101F7400002403E110E00E94AA042091FE2307EF4D
:101F840011E00E94AA042091ED230FE110E00E94C9
:101F9400AA042091FC2306EF11E00E94AA042091D8
:101FA4006A2308EF11E00E94AA042091F42309E0B7
:101FB40010E00E94AA042091F52303E010E00E949F
:101FC400AA042091F6230CE110E00E94AA042091B7
:101FD400FD230DE010E00E94AA042091092408E0EA
:101FE40010E00E94AA049ED208950E942C23A0E02F
:101FF400B0E000E0009300088CE491E012C080930C
:1020040026099093270900E61AEE0E94A301E9D15C
:10201400A017B10728F4D80180935F23909360231D
:1020240005968D3E02E0900750F300915F231091D6
:102034006023009326091093270947D43091602325
:10204400232F01E010E00E94AA0420915F2302E004
:1020540010E00E94AA04E4E00C943D230E9428238B
:1020640000E000930008009176230E94AA0180E01A
:1020740090E0A0E01DC0E6E8F3E200811181228136
:1020840033810E94F020A801B9012A013B01E2E852
:10209400F3E200811181228133810E94F020A201A8
:1020A400B3015ED1800F911F04E10E94AA01A395A0
:1020B400A53008F345E050E08C010E942720C801B8
:1020C400E091DA23F091DB23E81BF90BE65AFF4F8A
:1020D400E093DA23F093DB230091DA231091DB23DE
:1020E400093621E0120744F0EAEDF3E200811181A0
:1020F40008561140008311831091DB23112342F40D
:10210400EAEDF3E20081118108591E4F0083118327
:1021140009D2E8E00C9439230E942C23D80180E0F2
:1021240090E02AC00DE210E0AC010E94FB1FF80110
:10213400EA0FFB1FE83601E0F00714F0E856F1401F
:102144008F01212F220F220B322F0E94F02045E312
:102154005AEF6EE87CE30E94B0210E947B28AC0118
:10216400440F551F440F551FFA01E352FD4D0083E0
:102174001183228333830196883000E0900794F220
:10218400E4E00C943D230E942C23D80180E090E0ED
:102194002AC00DE210E0AC010E94FB1FF801EA0F17
:1021A400FB1FE83601E0F00714F0E856F1408F0118
:1021B400212F220F220B322F0E94F02045E35AEFE9
:1021C4006EE87CE30E94B0210E94A91FAC01440F79
:1021D400551F440F551FFA01E350FD4D0083118331
:1021E400228333830196883000E0900794F2E4E080
:1021F4000C943D230E942823D80180E090E034C051
:102204008D01212F220F220B322F0E94F020280152
:1022140039018C01212F220F220B322F0E94F02032
:102224004BED5FE069E47FE30E94B0210E947B28CC
:10223400A201B3010E94B021280139018D01212F8F
:10224400220F220B322F0E94F020A201B3010E9420
:102254004F210E94FD209C01220F331FF901E353FB
:10226400FD4D008311830196883000E0900744F20D
:10227400E8E00C943923B8014091FC2350E0890133
:102284000E94FB1F0D3B22E0120714F00CEB12E03E
:1022940023E22093010824E02093000800932A08F5
:1022A40010932B08609326087093270808950E94C2
:1022B4002C23D80104E00093000888E090E012C0C9
:1022C4004091FC2350E08C010E94FB1F00932A08DC
:1022D40010932B08A0932608B093270803E00E94CC
:1022E400AA010197813000E0900754F7E4E00C94D0
:1022F4003D23980103E2009301084091FC2350E040
:102304000AE010E00E94FB1F00932A0810932B0898
:1023140004E610E0A9010E94FB1F00932608109315
:10232400270804E00093000844E650E000915F238E
:10233400109160230E9427200E5F0E94AA0100E0F2
:102344000093000808958A93812F10E0D2DF00E300
:1023540015E70E94A301082F10E0CBDF89910895AF
:102364000E94411F40E050E064E672E40E94B02104
:102374000E94FD2008950E942823C801D9012A0142
:102384003B01A201B3012A013B010091E92310E0C2
:1023940020E030E00E94FB20A801B90182019301F2
:1023A4000E942922AC01BD010E944F21A201B30168
:1023B4000E94411F40E050E064E672E40E94B021B4
:1023C4000E94FD200B3520E0120714F00AE510E00E
:1023D400063A2FEF120714F406EA1FEFE8E00C9414
:1023E40039230E942C2380E090E000E00093220235
:1023F40000E00093010204E00E94AA01A0E0B0E022
:1024040019C00EE110E00E94A301E0E0F2E00081B7
:102414000860008300912B020023E1F301E00093A4
:102424002B020091120210911302801791070CF4F1
:10243400C8011196A43F01E0B0071CF300E100932A
:10244400010202E000932202835D9040992312F47A
:1024540080E090E042E050E08C010E942720E4E01C
:102464000C943D23E0E0F2E00081006100830091E0
:1024740033020023E1F301E0009333024091F82397
:1024840050E000911402109115020E940F20209137
:10249400012430E0220F331F220F331F020F131FBA
:1024A40008950E942C230EE210E0DAD2802F0FE26E
:1024B40010E0D6D2482F502F8A01212F220F220B51
:1024C400322F0E94F02040E04093010241E040930B
:1024D4000202E0E0F2E040814062408340913B022E
:1024E4004423E1F341E040933B02A801B90100E039
:1024F40010E02EEA33E40E942922C801D901009198
:1025040016021091170220E030E00E94FB20AC017B
:10251400BD010E94B0210E94FD200C521140E4E054
:102524000C943D230091DA231091DB23F5DD009117
:10253400DA231091DB2327DE08950091DA2310912A
:10254400DB23EADD0091DA231091DB231CDE4091CA
:10255400FF2350E008E710E00E94FB1F4BDE0091D0
:102564005F2310916023009326091093270908958F
:102574009A938A9301E010E00E946004902F80E017
:1025840002E010E00E94600410E0802B912B809305
:102594005F239093602305E010E00E946004902F75
:1025A40080E006E010E00E94600410E0802B912B94
:1025B4008093DA239093DB230EE010E00E94600402
:1025C400902F80E00FE010E00E94600410E0802B68
:1025D400912B8093E0239093E12300E110E00E948B
:1025E4006004902F80E001E110E00E94600410E09C
:1025F400802B912B8093E2239093E32303E010E05C
:102604000E9460040093F5230CE110E00E94600432
:102614000093F62304E110E00E9460040093E82391
:1026240003E110E00E9460040093002409EF11E02C
:102634000E9460040093F72307EF11E00E946004F6
:102644000093FE230CE010E00E9460040093FF233B
:102654000CEF11E00E9460040093F82302EF11E0F4
:102664000E9460040093022406EF11E00E946004BB
:102674000093FC230DE010E00E9460040093FD230E
:102684000AE010E00E946004802F90E00BE010E06C
:102694000E946004102F00E0802B912B80930E2465
:1026A40090930F2409E010E00E9460040093F42347
:1026B4000091F423093040F400E01091F423112335
:1026C40019F00060002341F001E00093F42321E0BD
:1026D40009E010E00E94AA040EE110E00E946004E8
:1026E4000093F3230EEF11E00E9460040093F123A2
:1026F4000DE110E00E9460040093F2230BE110E06E
:102704000E9460040093042408EF11E00E94600416
:1027140000936A230FE110E00E9460040093ED230C
:1027240008E010E00E9460040093092405EF11E022
:102734000E94600400930824EEE0F4E2008101604A
:1027440000838991999108950E942C23C801A9E0DE
:102754000091F623A01B06E51091612311230AF4CE
:1027640085C020916123322F330F330B10E02017E3
:1027740031070CF07BC04AE0009161230E94EB1FFB
:10278400402F4A5F00910E2410910F240E940920CB
:102794000170002309F06AC00091FE23013029F47E
:1027A4009C010CE115E267DD8DC00091FE2302302F
:1027B400B9F40091612305312CF49C0100E21EE47C
:1027C4005ADD80C0009161230B342CF09C010CEA8B
:1027D4001DE051DD77C09C0100E717E14CDD72C0BC
:1027E4000091FE230330B9F49C01C901ABE0B0E0D1
:1027F40000916123102F110F110B4AE050E00E9449
:102804002720A01BB10B04E115E0AD010E94FB1FC2
:102814009C0131DD57C00091FE23043081F49C01FA
:102824000EE610E040916123542F550F550B041B05
:10283400150B42E850E00E94FB1F1DDD43C09C01C4
:10284400C90100916123102F110F110B4AE050E0D0
:102854000E942720F801ED54FD4D418150E006E926
:1028640010E00E94FB1F9C0106DD2CC00091612337
:10287400002342F5B0E00091DE231091DF23A0177E
:10288400B10704F5A4E04CEE009161230E94EB1F14
:10289400A01B4A2F00910E2410910F240E9409209E
:1028A4000170002379F496958795009161230D3E7C
:1028B4002CF09C0100E21EE4DEDC04C09C0100EE6E
:1028C4001BEAD9DCE4E00C943D230E942C23809184
:1028D4005F23909160230196AC01652F660F660B10
:1028E400762F00E01CE62CED32E00E948E2048E0BA
:1028F40050E060E070E00E948E20C801D90148EEEB
:1029040053E060E070E08C019D010E948E2008502D
:10291400009305248B380EE3900700E0A00700E045
:10292400B0073CF001E00093012402E000930402AC
:1029340006C000E00093012403E00093040208E0D1
:1029440010E020E030E0AC01BD010E943B2040E7F4
:1029540050E060E070E00E948E2000937223109398
:10296400732345E000917223109173230E94032086
:1029740040E250E00E94FB1F0093722310937323E4
:102984004EE750E000917223109173230E940F20B0
:102994000093742310937523009172231091732371
:1029A400009370231093712346E150E000910124B9
:1029B40010E0401B510B00915F23109160230E9493
:1029C40027200093762310937723E4E00C943D238F
:1029D4000093E82310912002137E109320020A959D
:1029E400000F000F10912002102B10932002089565
:1029F400BFDD6BDF2091E2233091E3230091E023DC
:102A04001091E123FCD099DD0091E823E1DF0091EE
:102A1400F42332D20091092410E01195019510405D
:102A2400212F220F220B322F0E94F02043E353E385
:102A340065E672E40E9429220E94BE29A801B90118
:102A440000E010E020E83FE30E942922EFE3F1E2F6
:102A5400008311832283338301E00093EB230895E1
:102A640022E02093CA01F801049000E00093CA0117
:102A7400002D08959A938A9390E088E005C0082F6A
:102A840010E0EEDF900F83958631C8F3992309F4A3
:102A940093E0092F8991999108950E942D230BEEBB
:102AA40011E00E9460040F3F09F047C00CEE11E0F2
:102AB4000E9460040F3F09F040C0DCDFA02FF1DC6E
:102AC4008091E42320915D23820F20916C23820F57
:102AD400800F90E003C00E94C82793959817D8F3FD
:102AE4000E94C827802F853008F489E5282F0BEE33
:102AF40011E00E94AA042A2F0CEE11E00E94AA04FD
:102B040020E00DEE11E00E94AA0420E00EEE11E098
:102B14000E94AA0420E003EF11E00E94AA040E948C
:102B2400C827202F0AEE11E00E94AA040E94C82799
:102B3400202F09EE11E00E94AA04E3E00C943E2346
:102B44009C01A801CA01892F90E04F7F50708C012D
:102B54000E94FB1F080F191FC801840F951F0796B9
:102B6400982F80E00FEF10E0041B150BA8014F7F96
:102B74005070842B952B8C01C90108950E942C233D
:102B84000BEE11E00E946004B02FA0E00CEE11E007
:102B94000E94600410E0A02BB12B0DEE11E00E9406
:102BA4006004902F80E00EEE11E00E94600410E0BB
:102BB400802B912B8D01C4DF0817190781F45ADF8C
:102BC400202F30E00FEF10E08F7F9070081B190B5F
:102BD4002017310721F402E0009307240DC000916F
:102BE40007240D5F009307240091072402500093EB
:102BF400072401E000930724E4E00C943D230E94A1
:102C040026234801D90180E090E046C00DE210E09F
:102C1400AC010E94FB1FA801480D591D483601E074
:102C2400500714F0485651408D01212F220F220BDA
:102C3400322F0E94F020280139018A01212F220F0E
:102C4400220B322F0E94F0200801190145E35AEFAC
:102C54006EE87CE3800191010E94B0210E947B28F0
:102C6400A201B3010E94B021280139018D01212F55
:102C7400220F220B322F0E94F020A201B3010E94E6
:102C84004F210E94FD209C01220F331FF901E354C0
:102C9400FD4D008311830196883000E090070CF409
:102CA400B5CFEAE00C9437239A938A9320E030E07E
:102CB40000E010E0A4DF08E00E94AA0100916C2368
:102CC40010916D23043620E0120708F4AFC088EE9B
:102CD4009DEF00E010E000932A2410932B2408C0F9
:102CE400EAE2F4E2008111810D5F1F4F008311833A
:102CF40000912A2410912B24083621E012072CF588
:102D0400209143213091442100912A2410912B24B5
:102D140076DF03E00E94AA0100916C2310916D23D9
:102D240008171907E8F680916C2390916D230091A0
:102D34002A2410912B240093262410932724E09115
:102D44006C23F0916D23F29758F688EE9DEF00E026
:102D540010E0009343211093442108C0E3E4F1E21E
:102D6400008111810C5E1F4F008311830091432168
:102D740010914421083E27E012072CF520914321AD
:102D840030914421009126241091272438DF03E058
:102D94000E94AA0100916C2310916D230817190752
:102DA40090F480916C2390916D23009143211091B4
:102DB40044210093282410932924E0916C23F0915A
:102DC4006D237E9758F62091282430912924009170
:102DD40026241091272413DF0091282410912924FC
:102DE4000093E2231093E3230091262410912724D7
:102DF4000093E0231093E1233091E123232F0EE08D
:102E040010E00E94AA042091E0230FE010E00E9449
:102E1400AA043091E323232F00E110E00E94AA04C6
:102E24002091E22301E110E00E94AA0410E502E3EC
:102E34008ADA89919991089500EB0093010202E2E4
:102E44000093020203E00093040200910124013084
:102E540021F402E00093040203C003E0009304029F
:102E640003E00093200208E200932102E0E0F2E094
:102E74000081016000830895013051F401E010E8FD
:102E840000930E2410930F240AE00093E92308957D
:102E9400023051F40FE110E800930E2410930F2434
:102EA40008E00093E9230895033051F40FE110E89A
:102EB40000930E2410930F2403E00093E923089554
:102EC400043051F40FE510E800930E2410930F24FE
:102ED4000AE00093E9230895053051F403E010EC6F
:102EE40000930E2410930F2405E00093E923089522
:102EF400063051F40FED10E800930E2410930F24C4
:102F040000E10093E9230895073049F40FED18E92F
:102F140000930E2410930F2400E10093E9230895F5
:102F24000E942C23F89400E30E945C010091200687
:102F340003600093200600914006006F0093400652
:102F440000916006086300936006E0E4F6E0008107
:102F54000260008300916006066000936006E0E86A
:102F6400F6E000810460008308E10093900604E128
:102F74000E94AA01E4E8F6E00081046000830AEFFD
:102F840011E00E9460040F3F09F0F5C000EF11E06A
:102F94000E9460040F3F11F481E001C080E001EF62
:102FA40011E00E9460040F3F11F401E001C000E051
:102FB4008023882351F020E000EF11E00E94AA044E
:102FC40020E001EF11E00E94AA0400E00093232412
:102FD40005C0009123240395009323240091232406
:102FE400043008F0C3C000E00093222413C0FC01A5
:102FF400E658FD4F24918C0100541E4F0E94AA04F0
:103004000196893000E0900790F300912224039503
:1030140000932224009122240330D8F622E001E018
:1030240010E00E94AA042AE302E010E00E94AA042D
:1030340020E005E010E00E94AA0424EB06E010E082
:103044000E94AA0422E808EF11E00E94AA0420E0EA
:103054000EE010E00E94AA0420E00FE010E00E94BD
:10306400AA0420E000E110E00E94AA0420E001E1AB
:1030740010E00E94AA042FE003E010E00E94AA04DA
:1030840028E00CE110E00E94AA0421E004E110E031
:103094000E94AA0420E009EF11E00E94AA0425E09E
:1030A4000CE010E00E94AA0421E00DE010E00E9470
:1030B400AA0422E007EF11E00E94AA0421E00AE03A
:1030C40010E00E94AA0420E80BE010E00E94AA0489
:1030D4002FE20CEF11E00E94AA0421E009E010E0C5
:1030E4000E94AA0424E106EF11E00E94AA0420E051
:1030F4000DEF11E00E94AA0421E00EEF11E00E94FE
:10310400AA0420E002EF11E00E94AA0427E00DE1E6
:1031140010E00E94AA0421E00BE110E00E94AA043E
:1031240021E00EE110E00E94AA0420E005EF11E086
:103134000E94AA0420E00AEE11E00E94AA0420E200
:103144000EEF11E00E94AA0428E508E010E00E94B6
:10315400AA0421E003E110E00E94AA0421E00FE1A7
:1031640010E00E94AA0480E090E04BCF20E00AEF38
:1031740011E00E94AA040AEF11E00E946004009387
:10318400232400912324043040F000E000932324FE
:1031940020E00AEF11E00E94AA040DEF11E00E9462
:1031A40060040093222400912224033040F000E0C4
:1031B4000093222420E00DEF11E00E94AA0418DC01
:1031C40000912224002331F40091640608610093E5
:1031D400640617C000912224013059F4E4E6F6E0B5
:1031E40000810F7E0083E4E6F6E00081086000833E
:1031F40008C002E00093222400916406077E009335
:10320400640608EE1DEF0E94A30103E20093010887
:1032140000E00093000803E20093410901E00093F9
:10322400400908EE13E00093660910936709809142
:103234006A2390E08857904080936A0990936B09C1
:1032440001E00093000900915F2310916023009333
:1032540026091093270903E0009306090091A200B0
:1032640007600093A20007E00093400804ED11E01A
:10327400009366081093670801E0009346080E94D3
:103284008D0100919300043019F400E100932203AE
:10329400E1E4F6E000810860008303E00093A50800
:1032A4000FE60093A60802EF0093A70808E1009335
:1032B400A40800E10093A308E2EAF0E000810160C1
:1032C400008300E00093242400914406006F0093DF
:1032D40044060091240603600093240602E00E9441
:1032E400AA01AADD00E210E0BBDB00930C0201E2BC
:1032F40010E0B6DB00930D0202E0009322020E946C
:1033040086010E947F0119D9E4E6F6E00081046099
:10331400008300ED17E00E94591100EA1FE00E94AB
:10332400591100E41FE10E94591102E00E94AA0110
:1033340000ED17E00E94591100E00093000800918D
:103344007623102F03E0109F002D0E94AA01E4E6CB
:10335400F6E000810B7F008311DC78940091E82370
:1033640037DBE4E6F6E000810260008304E10E94BA
:10337400AA0101E00093EB2300E0009306240AE095
:103384000093F0230093EF2300E010E020E030E00E
:10339400EEEAF3E20083118322833383E2EAF3E269
:1033A40000831183228333830093622301E010E0BE
:1033B400009310241093112401E00093EE2300E005
:1033C4000093022408EA009368230093672305E22C
:1033D40010E00E947B1102E00E94AA0105E210E0C5
:1033E4000E947B1104E10E94AA01B2C001E0009393
:1033F400EE2300E610E00E947B1104E10E94AA0182
:1034040000E410E00E947B1104E10E94AA010091F3
:10341400122410911324043620E0120741F4E8E842
:10342400F6E0008103FD03C001E00093FB23E8E81C
:10343400F6E0008103FF1CC00091FB230130C1F4BE
:103444000AE00E94AA01E8E8F6E0008103FF10C048
:1034540000E810E00E947B1100E610E00E947B115E
:103464000AE00E94AA01E4E8F6E000810B7F0083F1
:103474000091FA23013041F400E00093FA2300E3C1
:1034840010E00E947B1110DC00910D24013089F4BE
:1034940000E000930D24E4E6F6E00081046000837C
:1034A40000E21EE40E94A301E4E6F6E000810B7F43
:1034B4000083809112249091132401968093122406
:1034C40090931324853301E290070CF441C000E08B
:1034D40010E0009312241093132400910824002375
:1034E400F9F000916723102F110F110B212F312FA9
:1034F4000E94F02043E353E365E672E40E9429222C
:103504000E94BE29A801B90100E010E020E83FE3D1
:103514000E942922EFE3F1E20083118322833383A3
:1035240000E000930008009144060F7000934406E5
:10353400E4E6F6E000810D7F008300916C23109196
:103544006D23083E23E0120718F401E00093EB23F7
:103554000091F9230023E1F300E00093F9230091A3
:1035640006240130D1F400E00093062400916B237B
:103574000B3370F001EF11E00E9460040395202FDB
:1035840001EF11E00E94AA0400E000936B2305C040
:1035940000916B23039500936B2304E11091F523B1
:1035A400011B00930A240091EE23013009F0D2C1DB
:1035B400E2E8F3E20081118122813381EAE9F3E256
:1035C4000083118322833383E6E8F3E200811181CF
:1035D40022813381E6EAF3E2008311832283338379
:1035E4000091F423043079F4EAE9F3E200811181D3
:1035F4002281338135952795179507950093DC2310
:103604001093DD2326C0E6EAF3E2008111812281D2
:1036140033810E94F020C801D901EAE9F3E2008174
:103624001181228133810E94F020EFE3F1E2408195
:103634005181628173810E94B021A801B9018C017A
:103644009D010E9493210E94FD200093DC2310938E
:10365400DD2300910A24102F110F110B2091DC237C
:103664003091DD23021713070CF033C100E00093FF
:10367400EF230091F02303950093F0230B3018F00F
:1036840001E00093EB23EEE9F3E200811181228152
:103694003381EAE9F3E24081518162817381401B05
:1036A400510B620B730B4083518362837383EAEA89
:1036B400F3E20081118122813381E6EAF3E2408161
:1036C400518162817381401B510B620B730B4083E8
:1036D400518362837383EAE9F3E2008111812281D9
:1036E4003381EAE9F3E240815181628173810E946E
:1036F4003B20C801D901E6EAF3E2408151816281AD
:103704007381E6EAF3E200811181228133810E9410
:103714003B20800F911FA21FB31F8C019D010E94AB
:10372400F0200E9449290E94FD2043E00E940920C4
:10373400009314241093152410911524112352F48A
:103744002EE130E000E81BEB0E943D1100E315E799
:103754000E94A3010091142410911524212F220FFB
:10376400220B322F0E94F0200E941A270E94FD2073
:1037740000936923E6EAF3E2008111812281338117
:103784000E94F020A801B901CA01DB01EAE9F3E2D1
:1037940000811181228133810E94F020AC01BD019E
:1037A4000E94BD11009361230091162410911724E7
:1037B4002091DC233091DD2302171307A4F4009138
:1037C4006123009363230091142410911524009322
:1037D4001024109311240091DC231091DD23009315
:1037E4001624109317240091612310916523011767
:1037F40024F40091612300936423009164230093D3
:103804006523009163230093662300936123009151
:103814006123075A0331F0F400916123102F110F33
:10382400110B20916823322F330F330B021B130B20
:1038340044E050E00E94272010916823010F009378
:1038440067230091672300936823009167230A95F7
:10385400009367238091DC239091DD2302968C01F1
:10386400212F220F220B322F0E94F0200E941A27B0
:103874000E94FD2010E00093DE231093DF230091CB
:1038840004241091F023011708F0DEC10091ED2308
:10389400002329F40EE110E00E94A613D5C1009183
:1038A400ED23013059F405E010E04091DE235091FE
:1038B400DF230E94FB1F0E94A613C6C10091DC23D4
:1038C4001091DD2315950795159507950E94A6136C
:1038D400BBC100E00093010800E000930008E4E4A9
:1038E400F6E000810D7F0083EAE9F3E200811181B3
:1038F40022813381EEE9F3E200831183228333834F
:10390400E6EAF3E20081118122813381EAEAF3E2FB
:10391400008311832283338300E00093692310E042
:10392400009316241093172400E010E00093102451
:103934001093112400936223009361230AE50093FA
:10394400642300E00093F0230091EF230395009398
:10395400EF237AC1E2E8F3E200811181228133810D
:10396400EAE9F3E20083118322833383E6E8F3E296
:103974000081118122813381E6EAF3E2008311831D
:10398400228333830091F423043079F4E2EDF3E2EB
:1039940000811181228133813595279517950795EB
:1039A4000093DC231093DD2326C0E6EDF3E20081CF
:1039B4001181228133810E94F020C801D901E2EDF6
:1039C400F3E200811181228133810E94F020EFE330
:1039D400F1E240815181628173810E94B021A8018A
:1039E400B9018C019D010E9493210E94FD20009346
:1039F400DC231093DD230091DC231091DD23212FA0
:103A0400220F220B322F0E94F0200E941A270E94BC
:103A1400FD200093DE231093DF2380910A24982F46
:103A2400990F990B42E050E00091DC231091DD23C3
:103A34000E942720801791070CF0D5C000E0009366
:103A4400EF230091F02303950093F023EEE9F3E2D2
:103A54000081118122813381EAE9F3E240815181BD
:103A640062817381401B510B620B730B4083518342
:103A740062837383EAEAF3E2008111812281338154
:103A8400E6EAF3E24081518162817381401B510B6C
:103A9400620B730B4083518362837383EAE9F3E21D
:103AA4000081118122813381EAE9F3E2408151816D
:103AB400628173810E943B20C801D901E6EAF3E2E6
:103AC4004081518162817381E6EAF3E200811181D0
:103AD400228133810E943B20800F911FA21FB31FBC
:103AE4008C019D010E94F0200E9449290E94FD2022
:103AF40043E00E940920009314241093152410918C
:103B04001524112352F427E030E004EF1EE70E944D
:103B14003D1100E41CE90E94A3010091F023093047
:103B240070F12091DE233091DF23220F331F08E947
:103B34001AE34091DC235091DD2355954795559523
:103B44004795041B150B0E943D11E6EAF3E2008140
:103B54001181228133810E94F020A801B901CA0198
:103B6400DB01EAE9F3E200811181228133810E94C1
:103B7400F020AC01BD010E94BD11009361230091AE
:103B84001624109117242091DC233091DD23021791
:103B94001307A4F400916123009363230091142478
:103BA4001091152400931024109311240091DC2308
:103BB4001091DD230093162410931724009163239E
:103BC400009361230091142410911524212F220FB6
:103BD400220B322F0E94F0200E941A270E94FD20FF
:103BE4000093692331C000E000930008EAE9F3E29E
:103BF4000081118122813381EEE9F3E20083118394
:103C040022833383E6EAF3E2008111812281338146
:103C1400EAEAF3E2008311832283338300E010E0B5
:103C2400009316241093172400E010E0009310244E
:103C3400109311240093692300E00093F023009172
:103C4400EF2303950093EF230091EF23003F41F00E
:103C540010E00091F023003F19F010601123A9F047
:103C640000E010E0009310241093112400936223C9
:103C74000093612300E00093692310E0009314246F
:103C84001093152401E00093EB2300916123102F7E
:103C9400110F110B009318241093192480911024F0
:103CA4009091112403968C01212F220F220B322F85
:103CB4000E94F0200E941A2740E050E060E87FEB69
:103CC4000E944F210E94FD2000931A2410931B246C
:103CD400E091DC23F091DD2337972CF00091182438
:103CE4000093622309C000916223102F110F110B5E
:103CF4000093182410931924E091DC23F091DD2320
:103D04003B970CF4ABC040911A2450911B240091B2
:103D14001824109119240E94272042E050E00E94A8
:103D2400272000930C2480916323982F990F990BDB
:103D340000916523102F110F110B801B910B03961B
:103D44008C01212F220F220B322F0E94F0200E947F
:103D54001A270E94FD2000931C2410931D24009117
:103D64000C24102F110F110B40911C2450911D2471
:103D74000E94272000930C240091182410911924E8
:103D8400063520E012073CF042E000910C240E942A
:103D9400EB1F00930C240091182410911924809196
:103DA400052490E0C296081719079CF00091052499
:103DB40010E0015C1F4F2091182430911924021740
:103DC40013073CF042E000910C240E94EB1F009387
:103DD4000C2410911B2411231AF400E000930C24EA
:103DE40000910C2400231AF400E000930C240091A9
:103DF4000C240B301CF00AE000930C2400910C24DA
:103E0400102F110F110B20913E21322F330F330B42
:103E1400021B130B42E050E00E94272010913E2128
:103E2400010F00930C2400910C2400933E21009177
:103E34000C2400933E210091182410911924209100
:103E44001A2430911B24020F131F012B19F400E0D4
:103E540000930C2400910C2400930B24E8E8F6E072
:103E6400008100FDD4CA0091EE23013009F0BECADE
:103E740000E00093EE23BDCA00008895FECF0E94A7
:103E84002823C801D9012A013B015CD057D071F421
:103E94008201930153D051F401E2ECE2F4E2008395
:103EA40041830FEF1FEF2FE73FE73DC044D0A2014E
:103EB400B3010E944F21AC01BD0140D061F442D056
:103EC4003AD00E94CA220BED1FE029EC10F43FE324
:103ED4002AC03FEB28C0A201B3012DD00E942922A1
:103EE400080119012FD0820193010E94B22223D02C
:103EF400A0F41CD050F424D0A801B9010BED1FE0AC
:103F040029E430E40E9493210EC01AD04BED5FE007
:103F140069E470EC0E944F2106C008D010F410D060
:103F240002C00ED03058E8E00C9439230E94CA2213
:103F34008001910108958C019D0108950C94A8229B
:103F44000C94DF2740E050E060E070E008953F7794
:103F540041E00C947E2803E20DBF01E20EBFC0E0F5
:103F6400D1E20E949D27002311F00E9461280E9443
:103F740092170E943E1F0C943E1F0D01DA0140E08F
:103F840050E060E070E00E94A82239F400E010E004
:103F94004D934C9320E030E00CC0B901660F771FBD
:103FA4007E57572F550F550B7D935C932F773078A1
:103FB4003F63D00108950024E8E0EA9532F0001F41
:103FC400001C0416D0F3041AF8CF001F402D0095EE
:103FD4000895FF27442312F4F1604195002312F45D
:103FE400F09501950E94DD1FF0FD0195F1FD4195CD
:103FF4000895149F102D059F100D049F002D110D81
:1040040008954A951AF016950795FBCF08954A9599
:104014001AF015950795FBCF089500241124EFE0BD
:10402400001F111F001C111C0416150610F0041AA1
:10403400150AEA95AAF7001F111FA0010095109513
:1040440008955195419550400895FF27552312F442
:10405400F160F7DF112312F4F09507D00E940F20CE
:10406400F0FD03D0F1FDEDCF0895119501951040B9
:1040740008952224349F302D259F300D169F300D36
:10408400079F300D249F202D310D159F200D311DCC
:10409400069F200D311D149F102D210D321D059FEB
:1040A400100D211D321D049F002D110D221D321DE6
:1040B40008954A952AF03695279517950795F9CFCF
:1040C40008954A952AF03595279517950795F9CFC0
:1040D4000895002411241001E0E2EA9592F0001FF3
:1040E400111F221F331F001C111C221C331C041619
:1040F40015062606370688F3041A150A260A370A0F
:10410400ECCF001F111F221F331FA001B101009526
:104114001095209530950895FF27772312F4F160C8
:1041240015D0332312F4F09509D00E946B20F69534
:1041340008F404D0F69508F409C008953095209544
:10414400109501951F4F2F4F3F4F0895709560951F
:10415400509541955F4F6F4F7F4F0895FF2711246E
:1041640077FB660F771F089409F4771F679517F894
:10417400EE27002437FB220F331F089409F4331F62
:10418400279507F8089527FD0EC0EE0F001F111F95
:10419400221F3A953230B8F7332319F427FD31E062
:1041A40002C027FF30E0E03821F400FF08940EF449
:1041B40088940F4F1F4F2F4F3F4F323038F4332323
:1041C40019F427FD31E002C027FF30E03F3F29F01A
:1041D400220F000C379527950895ACC0032E0020BC
:1041E40012F40E94A020E02F012F122F232F3EE96A
:1041F400D1CF0024F8CFBCDF432F4F5748F04F31C5
:1042040048F007FC91C03FE72FEF1FEF0FEF089531
:1042140033278CC0322F212F102F0E2F4F51419551
:104224000E945B2007FE08950C94A020F901EE0F74
:10423400FF1F37FBFF3F31F0EF2BE12BE02B88947E
:10424400B8940895E02BE12B21F008949894B89445
:1042540008959894889438940895FB01EE0FFF1FF5
:1042640077FBFF3F31F0EF2BE52BE42B8894B894D8
:104274000895E42BE52B69F3E8CFEFDF68F021F430
:104284003723262F8A010895372FFBCFE6DF20F04E
:104294000BF008957327EAF751C0C8DFE8F3B3F3CE
:1042A40061F3DBDFC8F383F3A1F358DF4017510751
:1042B4006207730731F4011411F10024E89488941F
:1042C4002BC078F0332E372F732D322E262F632DEB
:1042D400312E152F532D302E042F432D302C012C2D
:1042E400132C371739F0669557954795F795E040A5
:1042F4007395F7CFE7FBEE0FE0E010246AF0EF0FC1
:10430400041F151F261F60F4279517950795E79539
:1043140008F4689433953ECFEF0B040B150B260B72
:1043240039CFE0E87E27B9CF302D30782227112706
:10433400002708953FE7302920E8F9CF3FEF2FEF1A
:10434400F6CF8BDFD8F3D1F370783727089585DF64
:10435400A8F3A3F3F9CF3078372793CF67DF70F34F
:1043640083F3A9F37ADF50F3B3F3A9F3F7DE01245F
:10437400E8943F57E040370FEF1F12F0D9F603C01F
:104384003A3E90F26894E0E00A92AA933A93AA27FC
:10439400332422243327049FF001059FF00D712D4F
:1043A400731F149FF00D711D221C069F700D211C9C
:1043B400331C159F700D211C331E249F700D211C6E
:1043C400331E169F200C311CAA1F259F200C311C64
:1043D400A31F269F300CA11D39915EF43395A69539
:1043E400379427947795F795E79533953130BCF357
:1043F40016C0AA2322F0332351F4339510C0339509
:1044040071F4A991099096CFA7FD09C03A95EE0FD2
:10441400FF1F771F221C331CAA1F3230A8F7E89411
:10442400FE2B09F068942A2F8101E72FA9910990A6
:10443400BACE13DF10F00BF087CF80CF0EDFE9F395
:10444400E0F3032E072670CF032E072673CFEEDE8C
:10445400A0F37BF399F301DF80F39BF3A9F37EDEF2
:10446400012427FD06C0000F111F221F3150E04018
:10447400F8CF67FD06C0440F551F661F7150F0400A
:10448400F8CFE894371BEF0B3158EF4F2AF0EE23A7
:10449400E9F63F3FD9F203C03A3EA8F26894E0E05F
:1044A400F0E01124139440175107620738F031509B
:1044B40008F46894000F111F221FEE1F041B150B34
:1044C400260BEF0B000F111F221FEE1F0A9279E13A
:1044D4007A95AAF0041715072607EF0730F0041B96
:1044E400150B260BEF0B089401C08894111C221C99
:1044F400331C001C000F111F221FEE1FE9CFF0F91F
:10450400E894E22BE12BE02B09F0689406943794AD
:1045140027941794E79508F468947395B9F3099070
:10452400332311F0F0FF09C0369427941794E795CC
:1045340008F4689433953130BCF3012D122D232DEA
:1045440032CE8BCE98940895189408956FDED0F3EC
:10455400C1F383DEB8F30417150726073707089558
:104564007CDEA0F063DE90F029F0E32FE7273AF435
:104574007317089572DE51F04EF0089408950417ED
:1045840015072607370719F016F4B8F78894089525
:1045940064DEE0F34BDED0F3E7DFC0F30894089564
:1045A4007591659155914591159011FA2590359025
:1045B4000895F9DF041B10E003C0F4DF041B150B9E
:1045C40020E030E005C0ECDF041B150B260B370B95
:1045D400B8F010FC17C045910590E00FF11F0417C7
:1045E400100540E02407340758F436F404910024FD
:1045F400F101E01BF0090994E00FF11F25903590BB
:10460400F101099411F4D6F7F1CF31960EF03196F9
:1046140050E060E070E045914B3F48F089F34F3F34
:1046240029F04E3F11F07591659155914591041B08
:10463400150B260B370B39F318F3E7CFFA92EA92EE
:10464400DA92CA92BA92AA929A928A927A926A92C6
:104654005A924A92BA93AA939A938A930895FF849A
:10466400EE84DD84CC84BB84AA84998488847F808E
:104674006E805D804C80BB81AA8199818881F0E045
:10468400EC0FFD1FEF0108950E942023C1D37A018E
:104694005B016B018824992450D157D130F160E03B
:1046A40070E00E94A822D1F50989002309F449C0C9
:1046B4008E149F044CF40CEF80160FEF900624F038
:1046C40000E0088BE818F9080FEFE00EF01E0A89E5
:1046D4000023A9F100E0098B34C027D10E942922CC
:1046E40097D30AE0800E00E0901E47EB53E46AEB98
:1046F40071E52AD190F325D160E271E425D1A0F6C9
:104704000E94292285D301E0800E00E0901EF3CFA1
:104714000CD17CD306EF800E0FEF901E40E057EED5
:104724006BED7EE207D1A0F308D104D108F0BCCF31
:1047340060E271E46BD30FEF800E901EF5CF01E0C1
:104744000A8B0889002319F06624772444C0992031
:10475400EAF4DDD02701E0D06624772404C0D7D062
:104764000FEFE00EF01E4FD3861497041CF40E2DA9
:104774000F29A9F70FEF1FEF0419150980169106E9
:104784000CF473C077246624639425C034017194B7
:10479400619400E0700A1FC0DAD00E94FD20402E10
:1047A400212F220F220B322F0E94F020A801B901E1
:1047B400CED00E949321A801B90100E010E020E2CC
:1047C40031E424D3042D005DA3D0930101E0F6D29B
:1047D400232B09F4A1D0E614F704F4F6B2D060EA6E
:1047E40070E4B2D008F041C044244394C601019758
:1047F400FC0100810E3251F0040D00830A3329F4C8
:1048040000E300834424439401C044240197AE167A
:10481400BF0670F340FA4EF508890023B1F0C601D3
:1048240002C000830197A816B90658F4FC0102914E
:104834000E32FC01B1F732970081FC01008301972D
:10484400F1CF01E0800E941E0DC001E0C00ED41E15
:10485400C60105C0FC010291FC0100830197A81662
:10486400B906C0F301E3F50100830989002311F4BB
:1048740008C0C6D2F60102910033D9F30E3209F40E
:10488400BFD208890023C1F1F601019399203AF4BB
:104894000DE23FD09194819400E0900A02C00BE2B3
:1048A40038D0442455240AE0C00ED41C01E06FD251
:1048B40051D0405DF60141936F014CD04801012B6A
:1048C400A9F702E0401600E0500684F332018201A9
:1048D40017D02081830114D0E40DF51D3B9720836C
:1048E4000FEF400E501E01E0401600E050067CF72A
:1048F40006EFC00E0FEFD01E8601E3E10C943123C6
:10490400119501951040F601E00FF11F089500E3A1
:10491400F60101936F0108950E2D0F2919F40A89E8
:10492400002311F00EE2F5DF089549EF52E065E14E
:1049340070E508950CD00C94B22203D060E87FE3B4
:10494400089540E050E0089502D00C94CA228C01EE
:104954009D0108954AE050E084010C9427200E94B0
:104964002023EF97EF976A972A873B8748875987D1
:1049740068017B0100E00D830E8302C005D20ED2D4
:1049840029D2053249F00023C9F70D811E81EF9623
:10499400EF966A96E0E1B2CF0081053221F42BD282
:1049A400F3D105E2ECCF00E00C830B830A83098387
:1049B4003E0102E103D205E411E2088B198B06C023
:1049C4000981002311F40081098315D2FBD100521F
:1049D400B9F3035059F00850B1F3025019F00350E1
:1049E40049F00CC00A8103950A83EFCF0B8103952C
:1049F4000B83EBCF0C8103950C83E7CF00810A3244
:104A040079F4B6D1AD90BD90AFD1BB203AF4B19456
:104A1400A19400E0B00A0A8103950A83ECD114C082
:104A2400AA24BB244AE050E00DC021916F01850106
:104A34000E94FB1FA22EBB24A00EB11E00EDA00EEF
:104A44000FEFB01EC2D188F30A81002311F000E0F9
:104A54000C83B8D10E32F1F4CED1B4D10A3231F490
:104A640087D18D909D9080D1C6D117C08824992478
:104A74004AE050E0AAD188F421916F0184010E9498
:104A8400FB1F822E9924800E911E00ED800E0FEFE5
:104A9400901EF0CF88248A94982C80E093D10C54F3
:104AA40021F00C5131F0045039F481E0C80EA5D145
:104AB40003C001E0C00ED81E8DD1E4E8F2E00C94EE
:104AC400DB2280FB5EF44D815E81652F660F660BF1
:104AD40053D1408351836283638352CF2D813E81BE
:104AE4004BD1208331834CCF43D10D9111963CD1CE
:104AF4000A8B2E0103E14BD1FAC03AD16D907D901F
:104B040033D1062D072921F406E5602E01E2702E2B
:104B1400992022F400E1802E07E2902E80E090E0BC
:104B240001C00196F30101913F01002319F088159A
:104B34009905BCF368D12301919581959040680E45
:104B4400791ED5C00B81002331F0082D092919F4F1
:104B540099248824839405E611E2088B198B088133
:104B6400003739F405D1F6D000E122D100E0098301
:104B74002BC0FDD01EF4F4D04BD101C0EBD0088182
:104B84000F3611F408E0F1CF053771F70AE0EDCFE5
:104B9400EED04D915D9126F46D917D91E5D005C0E7
:104BA400E3D0652F660F660B762FCA01DB017723EE
:104BB4004AF40DE209839095A095B09581959F4F95
:104BC400AF4FBF4F0AE0F4D03E0107E9F7D02E0102
:104BD40007E9DDD0082F092B0A2B0B2B11F001E07C
:104BE40001C000E00F83082D092919F40F8100FF8B
:104BF40017C0FAD0E889F989E00DF11D0081F301AD
:104C040002933F01F1D004D1012B022B032B89F72E
:104C1400992032F40C81002319F0FDD001C0DFD0BB
:104C24008E0109561F4F91D0D4F30B81002309F450
:104C34005EC00F8100FF5BC00881083711F00835A2
:104C440049F4E1D0F30108810083DDD000E3F301EE
:104C540000834DC00F3609F04AC0F30100810033D0
:104C640009F445C000E302933F0141C081E008819B
:104C740002500883082D092939F49924882483943F
:104C840008C000E0088380E099201AF406E0802E32
:104C940099246ED065D055DE60E070E00E94B222A7
:104CA40028F44DE24983732F7058372F3E0142E1B7
:104CB400640E751E6A0C7B1C4B814A938A934A814D
:104CC4004A93B301A401E0DC28010C81002379F0AC
:104CD400A2D082013AD05CF482D0FBCF91D006E717
:104CE400602E01E2702E09E7402E01E2502E4201AF
:104CF40086189708A814B9041CF480E090E007C053
:104D040090D0A818B90810E0A01AB10AC5010A8108
:104D1400002321F401C03FD00197EAF70981002361
:104D240039F032D004C030D0F30101913F0136D0C4
:104D34000FEF800E901EBAF70A81002309F420CEEB
:104D440001970AF41DCE27D0FBCF061917090815C1
:104D5400190508958D919D9107D0A0E0B0E00895C4
:104D64000D911D912D913D91A083B183089580FBF8
:104D7400F701A081B1810895F701A081B1810D915E
:104D84001D91F2DFF8010895288539850895400EB4
:104D940000E0501E08952885398500E2EA85FB85E8
:104DA40009950D811E810F5F1F4F0D831E8308958A
:104DB40010E00C871D871E871F870895600E00E092
:104DC400701E0895F60100810895F60100810053D4
:104DD4000A300895F60101916F010883089500E3F4
:104DE400F30102933F0108954C855D856E857F85AF
:104DF400AEDD0C946B2001E0C00E00E0D01E0895DF
:104E04000FEFC00EFBCF0FEF600EDACF0E94B02180
:104E1400C801D901089505D010E04501801A910A0E
:104E240008950981002311F001E0089500E0089538
:104E34000E942423229741E050E060E070E00E9449
:104E4400B22260F440E00E94A82221F402E26BD076
:104E54003FEF5FC001E267D03FE75BC0AE010E9455
:104E6400BF1FC801D90143EF54E065E37FE30E940B
:104E7400B22268F437FBAA0FBB1FB395B695A7956A
:104E8400B7F908811981015010400883198340E063
:104E940050E060E87FEB43D02801390140E050E066
:104EA40060E87FE33CD0A801B901820193010E942C
:104EB4002922C801D901A801B9012FD0280139013B
:104EC4000881102F110F110B212F312F0E94F02078
:104ED40048E152E761E37FE320D04801590142E20F
:104EE40052E964ED7EE38201930117D04DED5BE955
:104EF4006AE27FE316D0A201B3010FD044E050E090
:104F040060E070E40ED0AC01BD0107D0A401B5018E
:104F140008D02296ECE00C9435230C94B0218C013B
:104F24009D010C944F21ECE2F4E2008351830FEFD6
:104F34001FEF2FE7089501E008950E942C23C80174
:104F4400D9011A013F7740E856E968E17BE40E9401
:104F5400CA2238F416D0B38300E010E020E030E039
:104F64000DC03B2F0E94FD200E94F0200AD0338305
:104F7400A801B9018C019D010E949321E4E00C94E5
:104F84003D23F10100831183228308954DE65EE4FD
:104F940066EC71E4EAE7F1E2008111812281338158
:104FA4000E943B20075C1F4C2F4F3F4F008311830F
:104FB4002283338389011F7708950E942023C80127
:104FC400D901BF7741E050E060E87FE33B2F0E94C6
:104FD400B22270F440E00E94A82229F40BED1FE0F5
:104FE40029E43FE350C0CC24DD24EE24FF241CC07C
:104FF4000BEDC02E0FE0D02E09E4E02EF72E40E09A
:105004007FEB082F48D02801390140E050E060E8E8
:105014007FE38C019D013FD0A801B9018201930176
:105024000E942922C801D901AC01BD018C019D0156
:105034002DD02801390144E25FEF6BE27CEB26D0EE
:1050440048E854E466EA7EE328D048E150EC6FE394
:1050540070E423D045EB1CD0480159014AEE54EBCF
:1050640066E870E48201930118D046EB11D0A801E0
:10507400B901840195010E942922AC01BD0106D029
:10508400A601B70108D0E0E10C9431230C94B021BF
:105094005DEF68E670E40C944F21FDDFA201B301DB
:1050A400F5CF20E006D0E9F70895259102D0E9F77D
:1050B40008952D9301501040202F212B08958AE844
:1050C40094E5FC0105911491FC013296A591B491EB
:1050D400FC01349625913491422F432B19F0F901A8
:1050E400E4DF01C0DEDF069614E58639910748F354
:1050F400089540E00C947E280E9428232897802F4E
:10510400B32F442E40E050E060E070E00E94B222F1
:1051140010F401E001C000E0000F400EBF7743E847
:1051240059EF62E27FE3082F3B2F80D076D041E035
:105134005CEF6FE777E40E94CA2288F5AE010E9413
:105144009F276BD0042D10E06BD0488159816A8170
:105154007B8172D0088319832A833B83AE014C5F21
:105164005F4F2A0140E050E060E87EE35FD0A20197
:105174000E949F2740E050E060E870E40C811D81AC
:105184002E813F8153D0A801B901088119812A8158
:105194003B810E9493210E94FD20402E0CC00E945E
:1051A400FD20602E3DD0A801B9018C019D0133D0B2
:1051B400460C03E0402240FA3EF4AC01BD0100E09D
:1051C40010E020E83FE327D002E0401608F0B05892
:1051D4008C019D0129D0280139014BEF57ED6EE177
:1051E40079E324D045E656E269E97BEB21D048E532
:1051F40054E363EA7DE31CD041EE5DE565E27FEBB9
:1052040017D04BED5FE069EC7FE316D00DD0289604
:10521400E8E00C9439230E949321C801D901089530
:1052240020E030E00C94FB20AC01BD010C94B021D3
:1052340003D0A201B301FACF0C944F211B2F6A2F84
:10524400F901A081B181AD014F5F5F4F408351836C
:105254000C93A62FB12F0895BA93AA9324970A8387
:105264001B8389019E012A5F3F4F28833983BE0136
:10527400AE014E5F5F4F20E239E20E94B12420E08C
:10528400AA81BB812C932496A991B99108950E9477
:10529400242322974801590141E050E060E070E086
:1052A4000E94B22298F440E00E94A82229F400E06F
:1052B40010E020E030E04EC001E2ECE2F4E20083D2
:1052C40051830FEF1FEF2FE73FE744C0AE010E9469
:1052D400BF1FC801D90145EC53E062E47FE30E949B
:1052E4004F214AE151E562E17FE33BD0A801B901D6
:1052F4008C019D013BD0402E088100FF14C00A950B
:105304002DD0802F43EF54E065EB7FE3042D0E9402
:10531400B02137FB220F331F380F3695279537F905
:10532400C801D9010BC01AD0842D912FD90137FBA4
:10533400AA0FBB1FB00FB695A795B7F940E050E090
:1053440060E87EE38C019D010CD0AC01BD018401B9
:1053540095010CD02296ECE00C94352342E00C9499
:10536400EB1F0E94B0212801390108950E942922CF
:10537400A201B3010C944F210E9426232497B32F3A
:10538400992440E050E060E070E00E94B22288245A
:1053940008F48394BF7743E859EF62EA7FE33B2F35
:1053A40062D0AE010E949F276BD080FA442440F85B
:1053B40001E0402653D00E94FD2003700A9529F095
:1053C4000A9531F00A9531F007C04FD0939404C088
:1053D400842CFCCF4AD0842CAC01BD018C019D01EE
:1053E40042D0088319832A833B8344E556E768E463
:1053F40071EC39D040E759ED63E52DD0280139012E
:105404004DE354ED6EE872EC29D00E944F2148819F
:1054140059816A817B8127D045E15EED66E81BD026
:10542400A801B901820193010E942922AC01BD01A6
:105434001AD026D090FA36F4A801B9011CD00E94E3
:1054440029221ED080FA0EF4B0588C019D012496B6
:10545400EAE00C94372373E40C944F2108811981FA
:105464002A813B8108950C94B021AC01BD0103D085
:105474000E94932105C000E010E020E83FE3089576
:10548400C801D90108955A0024219654B0027E21FE
:10549400000025303564002530356600253033643E
:1054A400002530336420002530345800010AD7A386
:1054B400BC2C01303132333435363738394142432C
:1054C40044454600286E756C6C20706F696E746577
:1054D40072290030313233343536373839616263FA
:0C54E400646566003F3F3F0001000000CF
:0400000300000000F9
:00000001FF
